:020000040000FA
:040000006B303A28FF
:08000800A000030EA100831209
:1000100005191028831601178312B23081002B288E
:1000200083160113831203140B190310A80DA90DD5
:10003000AA0DAB0DAC0DAC16FF302C02031D2B2806
:10004000FA302B02031D2B2831152A08AF0029088E
:10005000AE002808AD008B100B11210E8300A00EFE
:04006000200E090065
:0C007400203084008001840A80300402E7
:10008000031C3C281230B0008B2183160C308505F0
:1000900087018312850187010730990000309A009B
:1000A000103083168E008312603083168F00831207
:1000B0000030831691009F008312C83083168100A0
:1000C000831231309000003083168C008312103080
:1000D0008B00D62181018E018F010B118B100B102B
:1000E0008C018B17812031198420B30B7F280310DA
:1000F00085190314B90DF030390203191021EF21CD
:10010000722864003210080031110130B7008B13DF
:100110002030370783169B001C141A088312A40092
:100120001030370783169B001C141A088312A30093
:10013000A6000230A6060030370783169B001C1469
:100140001A088312A200A7000130A7068B17321CE1
:10015000AF2822090339A200A309A409A50924088C
:100160002F02031D0A2923082E02031DDE28220860
:100170002D02031D0A2901303702031DC2283D1438
:100180003E149F2102303702031DC928BD143E14BE
:10019000A32103303702031DD0283D153E14A721AB
:1001A00004303702031DD728BD153E14AB2105309E
:1001B0003702031DDE283D163E14AF2126082E020D
:1001C000031D0A2927082D02031D0A2901303702C1
:1001D000031DED283D103E14B32102303702031DEC
:1001E000F428BD103E14B72103303702031DFB284D
:1001F0003D113E14BB2104303702031D0229BD11FD
:100200003E14BF2105303702031D09293D123E145B
:10021000C3210A29B70A06303702031808008728C5
:100220000130B600B300B400B500B7008501870106
:10023000B1138120B30B3C29031085190314B90DA8
:10024000F030390203196329B40B3C29013037021D
:100250000319C721023037020319CA2103303702BC
:100260000319CD21043037020319D021053037029C
:100270000319D3219630B400311D19293111321CD4
:1002800046292D090339AD00AE09AF092F1C1929E4
:100290008E018F010C1C19290C102E1E19298B138D
:1002A00020303707BB002F08BA00762110303707FF
:1002B000BB002E08BA00762100303707BB002D089E
:1002C000BA0076218B1785018701B70AB60106307F
:1002D0003702031C1929D62108003E1C08003E10D5
:1002E0001030BB003D08BA00762108008B133A0895
:1002F00083161C159A0083123B0883169B00553009
:100300009D00AA309D009C1464009C1884291C1137
:1003100083128B170800831610309B001C141A08D8
:100320008312BD00FF30D000D415D515D615D715D2
:10033000D815D915DA15DB15DC15DD150800D21036
:100340004E14CE100800D2114E15CE110800D21254
:100350004E16CE120800D2134E17CE130800D3103B
:100360004F14CF1008005210CE144E100800521136
:10037000CE154E1108005212CE164E12080052131E
:10038000CE174E1308005310CF144F100800303012
:100390008506080003308506080006308706080039
:1003A0002130870608001830870608003D184E14D3
:1003B0003D1CCE14BD184E15BD1CCE153D194E1654
:1003C0003D1DCE16BD194E17BD1DCE173D1A4F143B
:1003D0003D1ECF144E08D2004F08D30008008F08EE
:1003E000031908008F01D00F312BD00A521C072AA5
:1003F000541DFD29D4015416152AD41D022AD401F6
:100400005416152A541E152AD401D414152AD41CA6
:100410000C2AD4015415152A541D112AD401D415BF
:10042000152A541E152AD4015415D21C262A551DEE
:100430001C2AD5015516342AD51D212AD501551659
:10044000342A551E342AD501D514342AD51C2B2A1A
:10045000D5015515342A551D302AD501D515342A14
:10046000551E342AD5015515521D452A561D3B2AC5
:10047000D6015616532AD61D402AD6015616532A9F
:10048000561E532AD601D614532AD61C4A2AD60100
:100490005615532A561D4F2AD601D615532A561ED5
:1004A000532AD6015615D21D642A571D5A2AD70140
:1004B0005716722AD71D5F2AD7015716722A571E60
:1004C000722AD701D714722AD71C692AD701571567
:1004D000722A571D6E2AD701D715722A571E722A03
:1004E000D7015715521E832A581D792AD80158164C
:1004F000912AD81D7E2AD8015816912A581E912A71
:10050000D801D814912AD81C882AD8015815912AC4
:10051000581D8D2AD801D815912A581E912AD80124
:100520005815D21EA22A591D982AD9015916B02A47
:10053000D91D9D2AD9015916B02A591EB02AD901B0
:10054000D914B02AD91CA72AD9015915B02A591D86
:10055000AC2AD901D915B02A591EB02AD90159158A
:10056000521FC12A5A1DB72ADA015A16CF2ADA1D9C
:10057000BC2ADA015A16CF2A5A1ECF2ADA01DA1417
:10058000CF2ADA1CC62ADA015A15CF2A5A1DCB2ADD
:10059000DA01DA15CF2A5A1ECF2ADA015A15D21FEC
:1005A000E02A5B1DD62ADB015B16EE2ADB1DDB2A67
:1005B000DB015B16EE2A5B1EEE2ADB01DB14EE2A62
:1005C000DB1CE52ADB015B15EE2A5B1DEA2ADB0159
:1005D000DB15EE2A5B1EEE2ADB015B15531CFF2A9E
:1005E0005C1DF52ADC015C160D2BDC1DFA2ADC01F2
:1005F0005C160D2B5C1E0D2BDC01DC140D2BDC1CA2
:10060000042BDC015C150D2B5C1D092BDC01DC15BA
:100610000D2B5C1E0D2BDC015C15D31C1E2B5D1DF0
:10062000142BDD015D162C2BDD1D192BDD015D1654
:100630002C2B5D1E2C2BDD01DD142C2BDD1C232B24
:10064000DD015D152C2B5D1D282BDD01DD152C2B0F
:100650005D1E2C2BDD015D156D214E08D2004F086B
:10066000D3005008D1000C305405031D05120C3086
:100670005505031D85120C305605031D05100C3061
:100680005705031D85100C305805031D87100C30CD
:100690005905031D07110C305A05031D07100C30B6
:1006A0005B05031D87120C305C05031D07120C301F
:1006B0005D05031D871151080E0203188B2B1230A4
:1006C0005405031D051612305505031D85161230FD
:1006D0005605031D051412305705031D85141230ED
:1006E0005805031D871412305905031D07151230D4
:1006F0005A05031D071412305B05031D87161230BF
:100700005C05031D071612305D05031D8715FF30BC
:100710005002031908008F08031D080081205108AA
:100720000E02031C8B2B18305405031D05120630D6
:100730005405031D051618305505031D8512063096
:100740005505031D851618305605031D0510063086
:100750005605031D051418305705031D8510063076
:100760005705031D851418305805031D87100630E2
:100770005805031D871418305905031D071106304D
:100780005905031D071518305A05031D07100630BB
:100790005A05031D071418305B05031D8712063028
:1007A0005B05031D871618305C05031D0712063014
:1007B0005C05031D071618305D05031D8711063003
:0807C0005D05031D871508000B
:084000000200030006000200AB
:02400E00CC33B1
:10420000010078007A007C007E007B0079007F004E
:104210007D007A0078007E007C00FF00FF00FF0038
:104220000000F200F600FA00FE00F200F600FA00CC
:10423000FE00F200F600FA00FE00FF00FF00FF00A3
:10424000010005000500050005000900090009003E
:1042500009000D000D000D000D00FF00FF00FF0024
:10426000FF00FF00FF00FF00FF00FF00FF00FF0056
:10427000FF00FF00FF00FF00FF00FF00FF00FF0046
:10428000FF00FF00FF00FF00FF00FF00FF00FF0036
:10429000FF00FF00FF00FF00FF00FF00FF00FF0026
:1042A000FF00FF00FF00FF00FF00FF00FF00FF0016
:1042B000FF00FF00FF00FF00FF00FF00FF00FF0006
:1042C000FF00FF00FF00FF00FF00FF00FF00FF00F6
:1042D000FF00FF00FF00FF00FF00FF00FF00FF00E6
:1042E000FF00FF00FF00FF00FF00FF00FF00FF00D6
:1042F000FF00FF00FF00FF00FF00FF00FF00DD00E8
:00000001FF
